:1000000013C0189518951895189518951895189562
:10001000189526C11895189518951895189518953E
:1000200018951895189518958FE181BD87E181BDC8
:100030008FE58DBFCCEFE4E44E2E84E08EBFD3E09D
:10004000F3E05F2EEEEFF3E0A0E6B0E088278D93BB
:100050003197E9F7A6D66624E5E0F0E0A8E7B0E03E
:1000600091E08DDAE8EBF5E188D9E8E7F0E0D080BF
:10007000EE24FF24002745D898D8FF27EDE0A9E813
:10008000B0E05DDAE6E0F0E0A8E7B0E091E077DA32
:10009000ECEBF5E172D9E8E7F0E0D080EE24FF2444
:1000A00000272FD882D8FF27EDE0A4E7B0E047DA99
:1000B000E4E7F0E007D8E9E8F0E0FFD70CD9FF2744
:1000C000EDE0A9E8B0E03BDAE0ECF5E156D9E9E88B
:1000D000F0E0F3D700D9FF27EDE0A9E8B0E02FDA90
:1000E00080E288BB86EC87BB80E082BB8DE781BB6A
:1000F00080E085BB80E084BB3AD68CE09ED6E8EEFB
:10010000F5E12FD68FEB11E041D6E2EFF5E129D6EC
:10011000E1E0F0E03DD685E083BF89B7816089BF2B
:1001200080E985BF7894E1E0F0E0A8E7B0E091E0F5
:1001300026DA009178000F3F09F014C088E380931D
:100140007800E1E0F0E0A8E7B0E091E07BE706DAD4
:1001500080E080937800E2E0F0E0A8E7B0E091E092
:100160007BE7FCD9B59901C000D3E1E0F0E0A8E756
:10017000B0E091E004DAE8EBF5E1FFD8E8E7F0E081
:10018000D080EE24FF240027BCD70FD8FF27EDE056
:10019000A5E8B0E0D4D9E2E0F0E0A8E7B0E091E073
:1001A000EED9ECEBF5E1E9D8E8E7F0E0D080EE2419
:1001B000FF240027A6D7F9D7FF27EDE0A4E7B0E09A
:1001C000BED9E4E7F0E07ED7E5E8F0E076D783D863
:1001D000FF27EDE0A5E8B0E0B2D9E4ECF5E1CDD839
:1001E000E5E8F0E06AD777D8FF27EDE0A5E8B0E0D2
:1001F000A6D9E3E0F0E0A8E7B0E091E0C0D9E8EBF1
:10020000F5E1BBD8E8E7F0E0D080EE24FF2400273A
:1002100078D7CBD7FF27EDE0AAE7B0E090D9E4E0AC
:10022000F0E0A9E7B0E091E0AAD9E2E4F2E080E4EE
:1002300004D658E0C895802DFAD531965A95D1F755
:1002400004C00E1B11111B0A1B2091D5B59905C0C6
:10025000A1E8B0E0E8ECF5E175D5F8CFF894FFCF70
:100260000F921F922F923F924F925F927F928F92A6
:100270009F92AF92BF920F931F932F933F934F93F1
:100280005F936F937F938F939F93AF93BF93CF931E
:10029000DF93EF93FF938FB78F93789421D094D00F
:1002A00039D198D18F918FBFFF91EF91DF91CF918D
:1002B000BF91AF919F918F917F916F915F914F917E
:1002C0003F912F911F910F91BF90AF909F908F9072
:1002D0007F905F904F903F902F901F900F901895B8
:1002E00080EC87B9BB27A7E28C9183608C93AEE743
:1002F000B0E062D881E0809378000091780000340B
:1003000010F009F040C083ED86B9BB27A6E20C913E
:1003100006FB0EF001C0F9CFA6E6B0E084B18C93E5
:10032000A7E6B0E085B18C93A7E6B0E08C91A2E699
:10033000B0E08D9388278C9398E0A2E6B0E09DD63C
:10034000A2E6B0E00D911C91A6E6B0E04D915527D4
:10035000040F151FA2E6B0E00D931C93AEE7B0E0CA
:100360000D911C91A2E6B0E04D915C91040F151F18
:10037000AEE7B0E00D931C93A8E7B0E08C918F5FDF
:100380008C9309F0BACF93E0AEE7B0E081D6ECEC05
:10039000F5E1F3D7EEE7F0E0D190E080FF2400270D
:1003A000B0D603D7FF27EDE0ACE6B0E0C8D8E5E86B
:1003B000F0E088D6ECE6F0E080D64DD7FF27EDE000
:1003C000ACE6B0E0BCD80895AEE7B0E0F5D780EC7D
:1003D00087B9BB27A7E28C9184608C9381E08093DE
:1003E000780000917800003410F009F040C083EDEF
:1003F00086B9BB27A6E20C9106FB0EF001C0F9CF2F
:10040000A6E6B0E084B18C93A7E6B0E085B18C930A
:10041000A7E6B0E08C91A0E6B0E08D9388278C939E
:1004200098E0A0E6B0E029D6A0E6B0E00D911C91DE
:10043000A6E6B0E04D915527040F151FA0E6B0E0E9
:100440000D931C93AEE7B0E00D911C91A0E6B0E0D7
:100450004D915C91040F151FAEE7B0E00D931C9316
:10046000A8E7B0E08C918F5F8C9309F0BACF93E04E
:10047000AEE7B0E00DD6E0EDF5E17FD7EEE7F0E0D6
:10048000D190E080FF2400273CD68FD6FF27EDE0F7
:10049000A8E6B0E054D8E9E8F0E014D6E8E6F0E0E9
:1004A0000CD6D9D6FF27EDE0A8E6B0E048D8E4EDB9
:1004B000F5E163D7E8E6F0E000D677D6FF27EDE078
:1004C000A8E6B0E03CD8E5E8F0E0FCD5E8E6F0E0EE
:1004D000F4D5C1D6FF27EDE0A8E6B0E030D8ECE6D1
:1004E000F0E0F0D5E8E6F0E0E8D5E6D6FF27EDE06D
:1004F000A8E6B0E024D8E8E6F0E0DFD5E8ECF5E1E6
:100500003CD744D708F005C0A8E6B0E0E8ECF5E138
:1005100019D408958DE0CCD481E0CAD484E0C8D445
:10052000A4E3B3E0AF93BF93E8E6F0E0C6D5C6D44A
:1005300011E002E0BF91AF9154D7E4E3F3E0AC8166
:10054000BD81F8D7AC81BD8131D8AA81BB818C93A4
:100550008FE712E01BD4AA81BB810C91043009F013
:1005600003C0EAEFF5E1FDD3AC81BD81F4D3ECEF3C
:10057000F5E1F7D38FE71BE009D4EAE7F0E0A2D575
:10058000ECE6F0E09AD511D6FF27EDE0A4E7B0E065
:10059000D6D7A4E3B3E0AF93BF93E4E7F0E08DD503
:1005A0008DD411E002E0BF91AF911BD7E4E3F3E0FB
:1005B000AC81BD81BFD78FEB13E0E8D3AC81BD81A7
:1005C000CAD3EEEFF5E1CDD382E1481A8827580A65
:1005D00026960895BB27A7E28C91807F8C93BB273A
:1005E000A7E28C9182608C938CE986B900000000B0
:1005F0008895A6E6B0E084B18C93A7E6B0E085B11B
:100600008C93A7E6B0E08C91A4E6B0E08D938827A8
:100610008C9398E0A4E6B0E030D5A4E6B0E00D916C
:100620001C91A6E6B0E04D915527040F151FA4E6D6
:10063000B0E00D931C93E8EDF5E19FD6E4E6F0E021
:10064000D190E080FF2400275CD505D6FF27EDE0A0
:10065000A0E7B0E074D7E4EDF5E18FD6E0E7F0E095
:100660002CD5A3D5FF27EDE0A0E7B0E068D7ECEDEF
:10067000F5E183D6E0E7F0E020D5EDD5FF27EDE00A
:10068000A0E7B0E05CD7E8E6F0E01CD5E0E7F0E0FA
:1006900014D512D6FF27EDE0A0E7B0E050D7EAE787
:1006A000F0E010D5ECE6F0E008D57FD5FF27EDE0CF
:1006B000A4E7B0E044D7E4E7F0E004D5E0E7F0E0F9
:1006C000FCD4C9D5FF27EDE0A0E7B0E038D7E0E7DC
:1006D000F0E0F3D4E0EEF5E150D658D608F005C0CE
:1006E000A0E7B0E0E8ECF5E12DD3E9E7F0E0D08059
:1006F000EE24FF24002705D5A4E7B0E036D5E0E7D7
:10070000F0E0DBD4E4E7F0E0DDD440D608F401C04B
:10071000C19AE4EEF5E131D6E9E7F0E0D080EE24CD
:10072000FF240027EED441D5FF27EDE0A4E7B0E099
:1007300006D7E4E7F0E0C6D4E9E7F0E0D080EE24A5
:10074000FF240027DED4B8D5FF27EDE0A4E7B0E012
:10075000F6D6E0E7F0E0B1D4E4E7F0E0B3D416D6A3
:1007600010F009F001C0C198089581E0A1D381E0A3
:100770009FD381E09DD381E09BD381E099D38BE02F
:1007800097D3882783BFF3D2E0E0F6E1EAD28FEB7C
:1007900011E0FCD2EAE0F6E1E4D2E2E0F0E0F8D2E7
:1007A000BB27A6E38C9185FBDEF7E1E0F0E0AA85AC
:1007B000BB8591E0E4D6E2E0F0E0A885B98591E060
:1007C000DED6D5D2E2E1F6E1CCD280E0AA81BB81CF
:1007D0008C938FEB11E0DAD2E8E1F6E1C2D2A4E328
:1007E000B3E0EA85FB855CD6B4D2A4E3B3E0E88548
:1007F000F98556D6AED2ECE1F6E1B3D2AA81BB813F
:100800000C91003510F009F001C047C0E1E0F0E0C4
:10081000AA85BB8591E07BE7A1D6E2E0F0E0A88560
:10082000B98591E07BE79AD6E8EBF5E1A6D5EA85B4
:10083000FB85D080EE24FF24002763D4B6D4FF27A5
:10084000EDE0A5E8B0E07BD6ECEBF5E196D5E885E8
:10085000F985D080EE24FF24002753D4A6D4FF27A7
:10086000EDE0A4E7B0E06BD6E4E7F0E02BD4E5E8F8
:10087000F0E023D430D5FF27EDE0A5E8B0E05FD667
:10088000E4ECF5E17AD5E5E8F0E017D424D5FF27CC
:10089000EDE0A5E8B0E053D656C0B59947C084E175
:1008A00090E0F7D2B5993EC080E0AA81BB818C93DD
:1008B000AC81BD818C918F5F8C93A885B9858C911B
:1008C0008F5F8C93A885B9850C910A3009F009C017
:1008D00080E0A885B9858C93AA85BB858C918F5FB4
:1008E0008C93AC81BD810C910A3010F009F001C0ED
:1008F0000DC08AE0AC81BD818C93AA85BB858C91AB
:100900008F5F8C9380E0A885B9858C93AA85BB8581
:100910000C91063410F009F001C004C088E2AA85E9
:10092000BB858C9386EE90E0B4D20CC080E0AC81A5
:10093000BD818C93AA81BB818C918F5F8C9382E364
:1009400090E0A7D246CF80E0AA81BB818C93E3E000
:10095000F0E0AE81BF8191E012D6AE81BF810C91F3
:1009600044E614D6AA85BB850C93AE81BF810C9159
:1009700044E60CD6A885B9858C938FE711E006D2A2
:10098000A4E3B3E0EA85FB858BD5E3D1E4E2F6E1AD
:10099000E8D1A885B9850C910A3008F003C0E6E2D9
:1009A000F6E1DFD1A4E3B3E0E885F98579D5D1D1CB
:1009B00080E03DD28FEB11E0E9D1E8EBF5E1DDD449
:1009C000EE81FF81D080EE24FF2400279AD3EDD35F
:1009D000FF27EDE0AAE7B0E0B2D582DCEAE7F0E07D
:1009E00071D3ECE6F0E069D3E0D3FF27EDE0A4E7B4
:1009F000B0E0A5D5A4E3B3E0AF93BF93E4E7F0E0A4
:100A00005CD35CD211E003E0BF91AF91EAD4E4E3A0
:100A1000F3E0A881B9818ED5A881B9819CD1E8E2A3
:100A2000F6E19FD1AA81BB810C91003510F009F04D
:100A300001C008C0E3E0F0E0AE81BF8191E07BE758
:100A40008DD537C0B59928C084E190E022D2B59900
:100A50001FC080E0AA81BB818C93AC81BD818C9149
:100A60008F5F8C93AE81BF818C918F5F8C93AC81B3
:100A7000BD810C910A3010F009F001C009C08AE074
:100A8000AC81BD818C93AE81BF818C91875F8C934B
:100A900086EE90E0FED10CC080E0AC81BD818C93ED
:100AA000AA81BB818C918F5F8C9382E390E0F1D11E
:100AB00054CFE5E0F0E0AA85BB8591E060D5E6E0A3
:100AC000F0E0A885B98591E05AD551D1E0E3F6E18F
:100AD00048D180E0AA81BB818C93E8EBF5E14DD44D
:100AE000EA85FB85D080EE24FF2400270AD35DD35E
:100AF000FF27EDE0A9E8B0E022D5ECEBF5E13DD42D
:100B0000E885F985D080EE24FF240027FAD24DD362
:100B1000FF27EDE0A4E7B0E012D5E4E7F0E0D2D2A1
:100B2000E9E8F0E0CAD2D7D3FF27EDE0A9E8B0E0CA
:100B300006D5E0ECF5E121D4E9E8F0E0BED2CBD374
:100B4000FF27EDE0A9E8B0E0FAD4CADB3DDCA4E37E
:100B5000B3E0AF93BF93E8E6F0E0AFD2AFD111E0DE
:100B600003E0BF91AF913DD4E4E3F3E0A881B98104
:100B7000E1D48FEB11E00AD1A881B981ECD0ECE18E
:100B8000F6E1EFD0AA81BB810C91003510F009F09D
:100B900001C00FC0E5E0F0E0AA85BB8591E07BE7EE
:100BA000DDD4E6E0F0E0A885B98591E07BE7D6D416
:100BB0004AC0B5993BC084E190E06BD1B59932C091
:100BC00080E0AA81BB818C93AC81BD818C918F5FC9
:100BD0008C93A885B9858C918F5F8C93A885B985F6
:100BE0000C910A3009F009C080E0A885B9858C9382
:100BF000AA85BB858C918F5F8C93AC81BD810C9154
:100C00000A3010F009F001C00DC08AE0AC81BD814E
:100C10008C93AA85BB858C918F5F8C9380E0A8858F
:100C2000B9858C9386EE90E034D10CC080E0AC8125
:100C3000BD818C93AA81BB818C918F5F8C9382E361
:100C400090E027D14ACF93D080E0AA81BB818C93DA
:100C5000E6E3F6E186D0E4E0F0E0AE81BF8191E02A
:100C60008ED4AE81BF810C91033610F009F001C023
:100C700004C080E0AE81BF818C938FEB11E086D001
:100C8000AE81BF810C910A3008F003C0EAEFF5E1B4
:100C900068D0A4E3B3E0EE81FF8102D45AD0EEE342
:100CA000F6E15FD0AA81BB810C91003510F009F00C
:100CB00001C00BC0E4E0F0E0AE81BF8191E07BE7D2
:100CC0004DD485E083BF53D037C0B59928C084E1A7
:100CD00090E0DFD0B5991FC080E0AA81BB818C93E2
:100CE000AC81BD818C918F5F8C93AE81BF818C91E3
:100CF0008F5F8C93AC81BD810C910A3010F009F0AC
:100D000001C009C08AE0AC81BD818C93AE81BF81F6
:100D10008C91875F8C9386EE90E0BBD00CC080E016
:100D2000AC81BD818C93AA81BB818C918F5F8C93A8
:100D300082E390E0AED095CF80E1481A8827580A28
:100D40002C96089584E0C89531960D928A95D9F72E
:100D50000895A4E3B3E08D91882311F068D0FBCF10
:100D6000089507D3802D11F062D0FBCF089581E064
:100D700064D014D080E861C08FE7213039F08FEB68
:100D8000223021F08FE8233009F08FEC810F55C01D
:100D900088EE93E07ED03197D9F7089583E09927C4
:100DA00078C08AEF90E075D08E9A8D9ABF9ABE9ADD
:100DB0008A9A889A9098EF93FF93E5E1F0E05DD0EE
:100DC000FF91EF91929896989598C79AC69A929AA1
:100DD000EF93FF93E5E1F0E050D0FF91EF9192980F
:100DE00055D0929AEF93FF93E5E1F0E046D0FF9162
:100DF000EF9192984BD0929AEF93FF93E5E1F0E058
:100E00003CD0FF91EF91929841D0C698929AEF937F
:100E1000FF93E5E1F0E031D0FF91EF91929836D069
:100E200088E20BD08EE009D086E007D00895909A32
:100E3000829505D004D02AD008959098F9CF859551
:100E400010F4C69A01C0C698859510F4C79A01C0DF
:100E5000C798859510F4959A01C09598859510F4DA
:100E6000969A01C09698929AEF93FF93E5E1F0E08D
:100E700004D0FF91EF91929808953197F1F708957A
:100E8000689462F80895E89462F8089581E090E02B
:100E900000C0EF93FF93EE27E82BE92B31F0EAEF48
:100EA000F0E03197F1F70197D1F7FF91EF910895B5
:100EB0005A924A92480E8827581E08958DE207FDDF
:100EC0008D938F2D881F802F881F8F57082F689430
:100ED000F7F8802F87FF15C080958395082F80E352
:100EE0008D938EE28D93802F815228F080E38D9335
:100EF00099279C93089544270A95802F09F192D051
:100F00001FC0805230F09EE49D9381E48D939D93A9
:100F1000EFCF4427DF92EF92FF920F938FE1801B78
:100F200011F0082F7FD085D09EE29D930F91FF9006
:100F3000EF90DF9044270395003209F4D7CF27D0F4
:100F40003F93E4ECFFE038E12F2D1E2D0D2DFF2403
:100F5000EE24DD244427000F111F221F88F42F9256
:100F60003F9207D2102C05D2202C03D2302C01D274
:100F70003197410DD21CE31CF01C3F902F9001C013
:100F8000339631963A9539F73F9107D0B3CFDD0CC0
:100F9000EE1CFF1C0A95D9F70895002719E058D0D8
:100FA0008F93802B11F0039501C08F911A95B9F79B
:100FB000802F882309F49ACF8F91805D8D930A95B5
:100FC000D9F796CF0065CD1D80B2E60E4059730764
:100FD000A0ACB90350D6DC01286BEE009435770045
:100FE000CA9A3B0065CD1D00B2E60E00597307009A
:100FF000ACB90300D6DC01006BEE000035770000D1
:101000009A3B0000CD1D0000E60E000073070000B3
:10101000B9030000DC010000EE00000077000000D2
:101020003B000000F694E794D79447950A95D1F7D2
:10103000089500270DD08F9303958F2D8E298D292C
:10104000842BC1F78F91805D8D930A95D9F750CF8E
:101050001F930F93002710E2440FDD1CEE1CFF1CB2
:10106000001F802F9AE0890B10F0082F43951A95E6
:1010700099F7802F0F911F910895903041F00D91B5
:101080001C91000F111F9A95E1F71C930E93089580
:10109000903041F00D911C91169507959A95E1F7C6
:1010A0001C930E930895D094E094F09491E0D90E9F
:1010B0009927E91EF91E10950895D190E190F190BD
:1010C0000191089521913191419151910895102FED
:1010D00090E8FF0C001F0927990FF7941078652FEF
:1010E00090E8440F551F5927990F479560780038AD
:1010F0000895FF0C90E89027110F9795F794092F0A
:101100000895112707FB56F4D094E094F0940095CD
:1011100091E0D90EE11EF11E011F1FEF9FE1DD0CD2
:10112000EE1CFF1C001F07FD07C09A95C1F7EE24B7
:10113000FF24002799270DC09258D7FA56F4E3945C
:1011400040F40024F01C001D20F493950795F794BB
:10115000E794DE2CEF2CF02E110F9795092F10F449
:10116000689401C0E894F7F80895DD92ED92FD923D
:101170000C930895502F2D2D3E2D4F2D612F089546
:101180002DEC3CEC4CEC5DE366270FC096DFF2DF04
:10119000DD24EE2490E8F92E0FE307C093DF05C0AD
:1011A0002227332740E251E46627552351F10023DB
:1011B00081F18DDF71F11627005850580894050B06
:1011C00018F407FD03C025C007FD23C046953795D9
:1011D0002795F694E794D79422D0FF202AF0DD0CCF
:1011E000EE1CFF1C015073F09D2D969548F0DD20FC
:1011F0003AF4EE202AF491E0D90E9927E91EF91E5F
:1012000078CF07C09FE7092FF92A9FEFD92EE92E43
:101210000895DD24EE24FF240027112708959F92CE
:101220009924AA24BB2488E1D216E306F40628F008
:10123000D21AE30AF40A089401C08894991CAA1CE3
:10124000BB1CDD0CEE1CFF1C8A9571F7D92CEA2C17
:10125000FB2C9F9008953BDFE1F25038D1F2162726
:10126000005850580894051F12F418F4CBCF08F01A
:10127000D0CF0AD0FF202AF0BB0CDD1CEE1CFF1CD7
:1012800038CF0F5FFBF135CF9F929924AA24BB245E
:10129000992788E1990CAA1CBB1CDD1CEE1CFF1CC5
:1012A00030F4920EA31EB41ED91EE91EF91E8A95B3
:1012B00089F79F90089506DF0ADF503829F090E8FB
:1012C00069270CC00AF045D014CF5FE322273327EB
:1012D000442701C0F7DEFBDE5038B1F3003899F344
:1012E000902F951B8BF312F434D0FACF983118F06D
:1012F000222733274427983028F0232F342F4427E0
:101300009850F9CF992329F04695379527959A95C6
:10131000D9F7912F962742F014D0B0F6F794E794BE
:10132000D7940F5F8BF66ECF10D051F008F4BBDE70
:10133000FF2052F2DD0CEE1CFF1C0150CBF762CFF8
:1013400068CFD20EE31EF41E0895D21AE30AF40AFF
:101350000895DF92EF92FF920F931F93D22EE32E08
:10136000F42E052F162F6F915F914F913F912F9182
:101370000895C895319600200895FBDF202DF9DFF0
:10138000302DF7DF402DF5DF502D089507FB006865
:101390000EF40F7757FB50680EF45F7707FD02C01D
:1013A00057FF05C0D216E306F406050708952D156C
:1013B0003E054F055007089582E001C084E099275B
:1013C0009D938A95E9F7089599278D9193958823A0
:1013D000E1F7939511968C9311978E919A95D1F789
:1013E0000895EA2FFB2F00248D9103948E32E1F7AC
:1013F00011248D9113948823E1F71A94101640F468
:101400001197202F2119239580E38D932A95E9F7D1
:10141000113011F59927AE2FFF2FA00DB91FA00F86
:10142000B91F8C919C93853308F41CC031E08E91D8
:101430008E32E9F3830F8A3319F480E331E001C07F
:1014400033278C93AE1799F7332329F0AE2FBF2F94
:10145000BBDF81E3808308958827E00DF81FE00F4C
:10146000F81F80830895000F111F221F331F089556
:1014700000951095209530950F5F1F4F2F4F3F4FD0
:101480000895019110810EC0019111912191308137
:101490000BC00191108117FF05C03FEF2FEF04C073
:1014A000008111272227332737FF03C0E1DF8DE2B8
:1014B0008D93CF93DF93CF92DF92EF92AA24BB2438
:1014C000CC24DD24EE2440E2CAE0DD2755E093E39E
:1014D0008881890F87FD9F7083FD907F891B899389
:1014E0005A95A9F7C0DFAA1CBB1CCC1CDD1CEE1C46
:1014F0004A9551F7E894EFE0FF2782910ED0EB3048
:10150000E0F71EF068948A2D0CD088278D93EF9019
:10151000DF90CF90DF91CF910895982F829501D0E1
:10152000892F8F70805D26F0803309F408956894C8
:101530008D93089581918D938823E1F7089594E028
:1015400081918D939A95E1F70895E199FECFEEBBD5
:10155000FFBB3196089591E001C092E07B3751F4D2
:101560007FB7F894F2DF8D918DBBE29AE19A9A955C
:10157000C9F77FBF7727089591E001C092E0E5DFCA
:10158000E09A8DB38D939A95D1F70895FF93881BB8
:10159000F9E0001FFA9511F4FF910895881F841B4C
:1015A00018F4840F8894F5CF0894F3CF8FEF8395C8
:1015B0009D919923E1F708950000C84200007A4404
:1015C00000005041000000400000000000100046F4
:1015D000000000410000804448E19C410AD72340BC
:1015E0000000003F0000A040444320504F574552A8
:1015F000000020535550504C590020005600410027
:1016000020207777772E656C0000666C792E706CE1
:101610000000567265663D00322E000056202020E4
:10162000202020002E0030004120202020202000FB
:101630005661646A3D005057522054722E00570084
:00000001FF
